:100000000C9432050C9493050C9482080C9493057F
:100010000C9493050C9493050C9493050C94930500
:100020000C9493050C9493050C9493050C94F5157E
:100030000C9493050C94A8230C9493050C949305AD
:100040000C9493050C9493050C9493050C94FD2348
:100050000C9493050C9493050C9493050C949305C0
:100060000C9493050C9493050C9493050C949305B0
:100070000C949305520A540A600A600A600A600AE6
:10008000600A600A560A580A5A0A600A600A540A44
:10009000620A600A600A1C0A520A600A600A580A68
:1000A000600A600A600A600A600A600A5A0A520A14
:1000B0003E0A600A420A600A600A600A1E0A560A7C
:1000C000600A600A4C0A600A600A600A200A5E0A36
:1000D000600A400A600A540A600A600A500A440A28
:1000E000600A460A580A600A600A600A4E0A480A0C
:1000F000600A600A600A600A600A600A600A4A0AC6
:10010000600A220A600A600A560A600A600A5E0AE9
:10011000600A600A600A600A600A600A600A600A8F
:10012000600A240A600A600A600A4C0A600A600ACF
:10013000600A600A600A600A600A600A600A600A6F
:10014000260A600A280A2A0A600A600A600A2C0A3B
:100150002E0A300A600A320A340A600A600A600A0B
:100160005C0A360A600A3A0A380A3C0A600A600ADF
:10017000600A600A5E0A860A940AA00AA00A780A3F
:10018000A00AA00AA00AA00AA00AA00AA00AA00A1F
:10019000A00AA00AA00AA00AA00A7A0AA00A7C0A59
:1001A000A00AA00AA00AA00A980AA00AAF0A960A02
:1001B000A00AA00AA00AA00AA00AA00AA00AA00AEF
:1001C000A00AA00AA00AA00AA00A700A8C0A7E0A45
:1001D000900AA00A800AA00A840AA00A8E0A820A4B
:1001E000920A880A8A0AA00AA00AA00AA00AA00AFB
:1001F000A00AA00A720A740A760A9A0A9C0AA00A3D
:10020000A00AA00A9E0A7E0B9E0BAA0BCE0BDE0B49
:10021000EA0B060C1D0C400C5D0C0B0D370DB50DDB
:10022000E70DD10DF80D0A0E120E180E1C0E220E3F
:100230007E0E800E820E840EC40E8C0E8C0E8C0EE2
:10024000860E880E8A0E5B1482147A1582147A1533
:10025000CE14F1147A154815571598199819D01914
:10026000D0194B1A5F1C5F1C5F1C7F1A5F1C271A7A
:10027000271A191C5F1C2E1C4C1C007B4601020314
:10028000763A687F6577482B353B6978796439140D
:100290001E3C6A7A1D16041A1F3D6B061B070821B7
:1002A000203E6C2C19091715223F6D11050B0A1CF5
:1002B00023406E7E100D182425416F360E0C122738
:1002C00026427037380F33132D43717534322F2E79
:1002D00044727C7D28303174457351504A524D49E7
:1002E0002A5466594F5C5F4C4B4E62635A5D5E60A8
:1002F000295367585B56576147554842403E3C3A40
:100300003B456843413F3D2B357E697A790078143F
:100310001E7C6A7B1D16041A1F7F6B061B070821B3
:10032000204D6C2C19091715224A6D11050B0A1C5A
:10033000234C6E49100D182425516F360E0C1227D0
:10034000264F7037380F33132D52717534502F2EBE
:100350004E72397D283065314B735464586776018D
:100360002A773259745C5F66020362635A5D5E608D
:10037000295344575B565561474680291E1F20214B
:100380002223242526272D2E2A2B141A0815171C64
:10039000180C12132F302878041607090A0B0D0EBB
:1003A0000F33343579311D1B0619051110363738D6
:1003B0007D557A2C393A3B3C3D3E3F4041424353C8
:1003C000475F6061565C5D5E57595A5B62634648A1
:1003D000324445677B7F650301025250514F686983
:1003E0006A6B6C6D6E6F7071725800494C754A4D36
:1003F000734B4E767C777E7466547225303258206B
:1004000000623A25303458200065253032582000EB
:100410002146554C4C2120002146462120007725BD
:100420003032582000214353335F4630210A0021E7
:100430004353335F5245414459210A00214353320B
:100440005F45305F4630210A00214353325F46301A
:10045000210A00214353325F4530210A00214353D2
:10046000325F494E4954210A00214353315F4530E0
:100470005F25303258210A000A5B4F56525D20003A
:100480004C2575200053257520000A49443A253033
:1004900034582825732920004D6F7573653A206EF6
:1004A0006F7420737570706F727465640A005225E2
:1004B0007520005725752000572575200057257594
:1004C00020005825752000412575200049257520FC
:1004D000005B4348475D20000A5052543A253032B1
:1004E00058204953523A2530345820005B52535417
:1004F0005D20000A4552523A253032582049535265
:100500003A2530345820000A4B6579626F61726475
:100510002073746172742E0A000A55534220636F6F
:100520006E666967757265642E0A000A0A544D4B3F
:100530003A65343733653863652F4C5546410A0AAE
:10054000003403490042004D0020005000430020C9
:10055000006B006500790062006F0061007200644A
:1005600000200063006F006E00760065007200746A
:10057000006500720000000E0374002E006D002E56
:10058000006B002E0000000403090409027400043B
:100590000100A0320904000001030101000921113A
:1005A0000100012240000705810308000A09040137
:1005B000000103000000092111010001223600079B
:1005C00005820308000A0904020002030000000972
:1005D00021110100012222000705830320000107E9
:1005E00005030320000109040300010300000009C2
:1005F00021110100012239000705840320000112A6
:1006000001100100000008EDFEEE1B0100010200D8
:100610000105010906A101050719E029E7150025D3
:1006200001950875018102050819012905950575CF
:100630000191029501750391010507190029F7152C
:1006400000250195F875018102C00631FF0974A1EA
:10065000010975150026FF009520750881020976AD
:10066000150026FF00952075089102C0050109803C
:10067000A10185021601002637001A81002AB70061
:10068000751095018100C0050C0901A101850316B3
:100690000100269C021A01002A9C02751095018116
:1006A00000C005010906A101050719E029E71500A9
:1006B00025019508750181029501750881010508DC
:1006C000190129059505750191029501750391019F
:1006D0000507190029FF150026FF009506750881FA
:1006E00000C0636F6E73756D65723A2025303458A3
:1006F0000A0073797374656D3A20253034580A0006
:100700000A002530325820006B6579626F6172648F
:100710003A20004C45443A20253032580A002558EA
:100720003A2530386225730A000A202030313233EE
:10073000343536370A0064656C5F6B65795F6269D2
:10074000743A2063616E27742064656C3A2025300A
:1007500032580A006164645F6B65795F6269743A5C
:100760002063616E2774206164643A20253032581A
:100770000A003F00433E20004C25640A000A092D70
:1007800020436F6E736F6C65202D0A4553432F71A4
:100790003A09717569740A000A092D204D6167696B
:1007A00063202D0A643A0964656275670A783A091C
:1007B0006465627567206D61747269780A6B3A09C5
:1007C0006465627567206B6579626F6172640A6D3A
:1007D0003A096465627567206D6F7573650A763ACC
:1007E0000976657273696F6E0A733A09737461747E
:1007F00075730A633A09636F6E736F6C65206D6F72
:1008000064650A302D343A096C61796572302D3493
:10081000284631302D4634290A506175733A0962F1
:100820006F6F746C6F616465720A6E3A094E4B5259
:100830004F0A003F004E4B524F3A206F66660A0047
:100840004E4B524F3A206F6E0A0074696D65725FAD
:1008500072656164333228293A202530346C580A95
:10086000006B6579626F6172645F6E6B726F3A20C4
:1008700025580A006B6579626F6172645F69646C08
:10088000653A2025580A006B6579626F6172645F72
:1008900070726F746F636F6C3A2025580A00686F2E
:1008A00073745F6B6579626F6172645F6C656473AA
:1008B00028293A2025580A000A092D20537461740A
:1008C0007573202D0A004743433A20352E342E30CD
:1008D000204156522D4C4942433A20322E302E3080
:1008E000204156525F415243483A20617672333577
:1008F0000A004F5054494F4E533A204C5546412020
:1009000045585452414B455920434F4E534F4C4547
:1009100020434F4D4D414E44204E4B524F204B45AE
:10092000594D41505F53454354494F4E20424F4F1C
:10093000544C4F414445525F53495A450A00425571
:10094000494C443A20653437336538636520283292
:10095000323A30313A3133204E6F76203232203203
:10096000303230290A005649443A2030784645450D
:100970004428742E6D2E6B2E29205049443A203085
:1009800078316265652849424D205043206B657976
:10099000626F61726420636F6E766572746572292E
:1009A000205645523A203078303030310A004445E4
:1009B00053433A20636F6E766572742049424D202E
:1009C0005043206B6579626F61726420746F2055AB
:1009D00053420A000A092D2056657273696F6E2012
:1009E0002D0A000A6D6F7573653A206F66660A00FE
:1009F0000A6D6F7573653A206F6E0A000A6B657930
:100A0000626F6172643A206F66660A000A6B6579EC
:100A1000626F6172643A206F6E0A000A6D617472CF
:100A200069783A206F66660A000A6D6174726978A7
:100A30003A206F6E0A000A64656275673A206F6E2D
:100A40000A000A64656275673A206F66660A000AE2
:100A50000A626F6F746C6F616465722E2E2E2000B7
:100A6000433E200011241FBECFEFD4E0DEBFCDBF38
:100A700004B603FE41C08091A2039091A303A0910C
:100A8000A403B091A5038730904BA740B04BA1F5CC
:100A90001092A2031092A3031092A4031092A50334
:100AA00014BE0FB6F894A895809160008861809379
:100AB0006000109260000FBE1092010810920008B2
:100AC000E3E0F0E089E080935700E491E695E3707D
:100AD000E150E33040F4F0E0EE0FFF1FE85BFE4F23
:100AE0008081918102C080E090E1E0E0F0E8E81BC5
:100AF000F90BF695E795099511E0A0E0B1E0E6E283
:100B0000FCE402C005900D92AE34B107D9F723E0A2
:100B1000AEE4B1E001C01D92A23AB207E1F70E9433
:100B20007A110C9411260C940000FF93EF93E0913E
:100B30004E01F0914F01309709F00995EF91FF9127
:100B40000895FC018591803011F0EFDFFBCF08950F
:100B5000FF27E0E230E247FF0CC0419597FF09C054
:100B6000EDE26095709580959095611D711D811DD8
:100B7000911D27FF02C0219530E350E2AA27660F9E
:100B8000771F881F991FAA1FA41710F0A41B639535
:100B90005A95A9F7AA3008F0A95FA05DAF93F39525
:100BA000611571058105910541F7ED3211F4EF935F
:100BB000F395F21718F43F93F395FBCF8F91B5DFC0
:100BC000FA95E1F70895E991F9918591803021F046
:100BD000853219F0AADFF9CF089520E0E894559105
:100BE0005532C1F3503311F4689455915A3348F497
:100BF000505390F3220F022E220F220F200D250FAB
:100C0000F4CF0EF4219589919991533619F3533706
:100C100029F1533559F1BC0188279927E8945C36AE
:100C200021F48991999168945591543639F446EF9D
:100C30007EF077FF0DC08FEF9FEF0AC055374AE077
:100C400039F0583540E121F0523642E009F008957C
:100C5000FF93EF937DDFEF91FF91B7CFFF93EF937A
:100C6000FC0181918030B9F360DFFBCFFF93EF93FC
:100C700068DFF1CFDF93CF93CDB7DEB72596A3DF43
:100C8000CF91DF91089590915B01923081F0933084
:100C9000D1F0913031F5E72FF0E0B3E0EE0FFF1F18
:100CA000BA95E1F7E60FF11DE658FC4F17C0E72FA4
:100CB000F0E0A3E0EE0FFF1FAA95E1F7E60FF11DAC
:100CC000E650FD4F0BC0E72FF0E073E0EE0FFF1F83
:100CD0007A95E1F7E60FF11DE658FD4FE491E03813
:100CE00019F480E090E0089590E023E0880F991FC8
:100CF0002A95E1F72E2F207730E044E035952795AF
:100D00004A95E1F7820F931F54E0880F991F5A9577
:100D1000E1F7EF709C012E0F311DF901EE0FFF1F5F
:100D2000E050F8498591949108955998519A089501
:100D30005198599A08955898509A08955098589AE9
:100D400008955198599A85E08A95F1F7000089B184
:100D50008695817008955098589A85E08A95F1F7A4
:100D6000000089B181700895CF93DF93EC010E9458
:100D7000A106882341F0209731F085E08A95F1F7AC
:100D800000002197F4CFCE01DF91CF910895CF934A
:100D9000DF93C2E3D0E00E94A106811108C0209732
:100DA00031F085E08A95F1F700002197F4CFCE016C
:100DB000DF91CF9108952E9826982F9827980E941A
:100DC00095060E949E06E9E6F0E0808188608083B7
:100DD000E9980895E19AE99A0E9498060C949E0673
:100DE000E9980E9495060C949E06CF93DF932FB747
:100DF000F894C0910201D0910301CE01882781159A
:100E00009F4F19F080E09FEF02C08FEF90E08C2B96
:100E10009D2B90930301809302012FBFCE01992750
:100E20008F3F910581F5CD2FDD27C03FD10551F0D2
:100E3000CF3FD10509F451C080918F03C034D10553
:100E400099F407C080918F0380FF33C088E194E05C
:100E500004C080FF2EC080E194E09F938F930E9496
:100E60003A060F900F9025C080FF37C0DF93CF93D5
:100E700089E094E09F938F930E943A060F900F9021
:100E80000F900F902AC0CE018F6F019699F080913C
:100E90008F0380FF0CC0DF93CF9381E094E09F939A
:100EA0008F930E943A060F900F900F900F90CD2FC6
:100EB00001C0CFEF80918F0380FF0CC01F92CF93B2
:100EC0008AEF93E09F938F930E943A060F900F90C2
:100ED0000F900F908C2F90E002C08FEF9FEFDF916B
:100EE000CF910895CF93CAE1C15069F00E94F506F1
:100EF0008F3F2FEF920749F48FE99FE00197F1F7B9
:100F000000C00000F1CF8FEF9FEFCF9108951092B6
:100F1000540110925301109252011092510180E03D
:100F200090E890930101809300018FEF9FEF9093E1
:100F30000301809302010895EF92FF920F931F9394
:100F4000CF93DF93082F1092510180918F0380FF80
:100F50000CC01F920F938EE194E09F938F930E9499
:100F60003A060F900F900F900F90E9980E94950607
:100F70000E949E068FE891E00197F1F700C0000003
:100F80000E949B068FE891E00197F1F700C00000F6
:100F90000E94980680E197E20E94B406892B11F422
:100FA00081E084C0C0E0D0E0FF24F39410E0EE24A0
:100FB000E39490E59A95F1F7C8010C2E02C095953F
:100FC00087950A94E2F780FF04C0FE240E949E06E3
:100FD00002C00E949B060E94C706892B11F482E082
:100FE00065C082E390E00E94B406892B11F483E08F
:100FF0005DC02196C830D105E1F680E58A95F1F70C
:10100000FF2019F00E949E0602C00E949B060E94CB
:10101000C706892B11F484E049C082E390E00E9466
:10102000B406892B11F485E041C090E59A95F1F75B
:101030000E949E060E94C706892B11F486E036C0E6
:1010400080915201813109F447C082E390E00E940F
:10105000B406892B19F0C2E3D0E009C087E026C0AE
:10106000209759F025E02A95F1F7000021970E947A
:10107000AB068111F5CFCD2B11F488E017C00E948B
:10108000C706892B19F0C2E3D0E009C089E00EC081
:10109000209759F085E08A95F1F7000021970E948A
:1010A000AB068823A9F3CD2BB9F48AE080935101D4
:1010B000809151018061809351010E9498060E94A5
:1010C0009E06E19AE99A8FEF9FEFDF91CF911F91F2
:1010D0000F91FF90EF9008958FEF9FEF9093030192
:1010E000809302010E9487070E9498060E949E0634
:1010F000E19AE99ADF91CF911F910F91FF90EF90C4
:101100000C9472071F920F920FB60F9211242F9317
:101110003F934F935F938F939F9329B18091900357
:1011200040910001509101014115504819F48093FC
:1011300050010FC090915001891B833050F0809175
:10114000000190910101909354018093530180E23A
:10115000DDC0809100019091010196958795909353
:1011600001018093000120FF09C08091000190914E
:10117000010190689093010180930001809100012A
:101180009091010199278038910509F4F9C0A8F4DC
:101190008032910509F4F4C038F4009709F4F0C0E6
:1011A000409709F489C0A9C08034910509F4E8C0CA
:1011B0008035910509F480C0A0C0803C910539F1CB
:1011C00050F48039910509F477C0803A910509F00F
:1011D00094C084E64DC0803D910509F46DC0803E09
:1011E000910509F08AC080910001909101019093CE
:1011F0005401809353018091000190910101892F46
:101200009927909301018093000183E252C084E604
:1012100049990FC0882369F095E09A95F1F700008D
:101220008150F6CF882349F095E09A95F1F70000B8
:1012300081504999F7CF8111A3C08091000190910D
:10124000010190935401809353018091000190918A
:101250000101892F9927909301018093000182E277
:1012600028C0882379F095E09A95F1F70000815025
:10127000499BF7CF07C0882349F095E09A95F1F78D
:10128000000081504999F7CF81117AC08091000107
:10129000909101019093540180935301809100013A
:1012A00090910101892F992790930101809300016A
:1012B00081E28093520133C080910001909101013D
:1012C000909354018093530180910001909101010A
:1012D00097FF02C080E101C081E1809352018091BB
:1012E00000019091010146E0969587954A95E1F7B6
:1012F000909301018093000112C0809100019091B0
:101300000101909354018093530180E8809351012F
:101310008091510190E0982F88278F6F27C080918E
:1013200000019091010199278F3F910511F480EF01
:10133000EDCF809103018F3F31F0809102018F3F0B
:1013400011F080E4E3CF8091020190910301982F86
:10135000882790930301809302012091000130912E
:1013600001018091020190910301822B909303016E
:101370008093020180E090E8909301018093000146
:101380009F918F915F914F913F912F910F900FBE41
:101390000F901F901895CF93C82F8DEE0E949C0739
:1013A0008A3F910521F48C2FCF910C949C07CF910B
:1013B0000895E82FE695E695E695EF70F0E0E15A9E
:1013C000FE4F4081282F277081E090E002C0880FF7
:1013D000991F2A95E2F7242F30E028233923232B65
:1013E00011F4842B80830895E82FE695E695E69521
:1013F000EF70F0E0E15AFE4F2081382F377081E026
:1014000090E002C0880F991F3A95E2F7422F50E012
:1014100048235923452B19F0809582238083089512
:10142000482F50E0FA013397E138F10508F048C041
:10143000E65CFF4F0C940B2687E108958FE1089539
:101440008CE5089580E6089582E6089587E2089580
:1014500083E508958FE2089589E3089587E3089569
:101460008FE3089587E408958FE4089586E508954D
:101470008EE508958FE7089580E0089585E6089544
:101480008EE608958FE6089580E3089588E3089531
:1014900080E4089588E4089580E5089587E5089537
:1014A0008FE5089588E1089588E0089580E2089521
:1014B00080E1089589E108958DE6089588E2089510
:1014C0008F7708958FE00895CF93482F50E0FA0169
:1014D0007C97E834F105A0F5E554FF4F0C940B26FA
:1014E00085E53EC08AE53CC08BE53AC08CE538C056
:1014F0008DE536C08EE534C08FE532C080E630C061
:1015000081E62EC082E62CC083E62AC08FE628C082
:1015100081E726C082E724C084E722C085E720C097
:1015200087E71EC088E71CC08AE71AC08CE718C08E
:101530008FE716C080E714C089E712C08BE710C0A0
:10154000C82F1F928F9389E694E09F938F930E94F8
:101550003A060F900F900F900F908C2F01C084E5EA
:10156000CF9108950F931F93CF93DF930E94D623BB
:101570008C010E94F506EC01019631F4C8010E942D
:10158000EE23843F9140A8F3CE01DF91CF911F91CC
:101590000F9108950E94DB060C94EA0680918F0358
:1015A000816080938F03EFE5F1E0119281E0EF36E7
:1015B000F807D9F70895E82FF0E0E15AFE4F80814F
:1015C0000895EFE5F1E0119281E0EF36F807D9F7E1
:1015D0000895982F80915B01823048F092FB882714
:1015E00080F990FD826091FD84600C94CB09089590
:1015F000CF93DF9380915101882371F18091530142
:1016000090915401209151019F938F931F922F939A
:1016100083EF94E09F938F930E943A06809151014B
:1016200080750F900F900F900F900F900F9071F4A6
:1016300080915A018B3051F48CEE94E09F938F93FC
:101640000E943A0610925A010F900F901092510189
:10165000109254011092530180915201882309F491
:1016600040C09091520180915E019817D1F1809114
:10167000530190915401209152019F938F931F9297
:101680002F9388ED94E09F938F930E943A06809168
:101690005E010F900F900F900F900F900F9085FFAD
:1016A00004C09091520194FD06C084FF12C0809145
:1016B000520185FF0EC080915A018B3051F481EDAB
:1016C00094E09F938F930E943A0610925A010F90D4
:1016D0000F908091520180935E01109254011092FC
:1016E0005301E0915A018E2F90E08C30910508F063
:1016F0004FC3FC01ED5FFE4F0C940B260E94F006D9
:101700000E94D6239F938F938CEC94E09F938F93AA
:101710000E943A0610925B0110925D0110925C01EA
:1017200010925E010E94E10A0E9448190E94D6238D
:10173000909359018093580181E065C080915801D0
:10174000909159010E94EE23893E934008F420C3F2
:1017500082E031C00E9487070E94EA068FE99FE07D
:101760000197F1F700C000008FEF0E949C078A3FAD
:10177000910511F486E001C083E080935A010E9434
:10178000D6239F938F9387EC94E09F938F930E942F
:101790003A060F900F900F900F90FAC20E94F00639
:1017A0002E98269A2F98279A0E94D6239093590113
:1017B0008093580184E080935A01EAC280915801D5
:1017C000909159010E94EE23853F914008F4E0C2B8
:1017D00085E0F1CF2E9826982F9827980E948707AA
:1017E0000E94EA060E94D6239F938F9382EC94E096
:1017F0009F938F930E943A060E94D623909359019B
:101800008093580186E080935A01C3CF0E94F50669
:10181000019609F4BDC20E94D6239F938F938DEB4E
:1018200094E09F938F930E943A060E94D623909350
:1018300059018093580187E0E6CF8091580190913B
:1018400059010E94EE23853F914018F089E0809372
:101850005A010E94F506019609F49AC20E94D62305
:101860009F938F9388EB94E09F938F930E943A0607
:101870000E94D623909359018093580188E0C3CFEA
:1018800080915801909159010E94EE23853F91402B
:1018900018F089E080935A010E94F506019609F438
:1018A00077C20E94D6239F938F9383EB94E09F93FC
:1018B0008F930E943A0689E0A6CF80915201813130
:1018C000C1F082EF0E949C078F3F2FEF9207A1F09B
:1018D0008A3F9105A1F40E94B20A8F3F3FEF930720
:1018E00089F0D82FCC270E94B20A9E01282BC9016B
:1018F0000BC08DEF9FEF08C08FEF9FEF05C08EEFFD
:101900009FEF02C080E090E090935D0180935C01C6
:101910000E94D6239F938F938EEA94E09F938F9398
:101920000E943A0680915C0190915D010F900F90AA
:101930000F900F90009711F482E031C08F3F3FEF7E
:10194000930711F481E02BC08E3F2FEF9207A1F394
:101950008D3F3FEF930711F484E021C08F3F910545
:1019600059F488E994E09F938F930E943A0610926D
:101970005B010F900F901FC09C0125583B4A2230FD
:10198000310580F480EF0E949C078A3F9105A1F603
:1019900083E00E949C078A3F910571F683E0809363
:1019A0005B0109C0803B2FEB9207C1F388278115AB
:1019B0009F4BA1F3C1CF80915B01813049F0823010
:1019C00051F0833059F0843061F087E291E00BC030
:1019D0008BE191E008C088E191E005C08EE191E0E3
:1019E00002C08CE291E09F938F9380915D018F9371
:1019F00080915C018F938AE894E09F938F930E947B
:101A00003A068AE080935A010F900F900F900F9042
:101A10000F900F90BDC10E94D6239F938F9385E8AE
:101A200094E09F938F930E943A060F900F900F902F
:101A30000F9080915B01823029F0833039F488EF78
:101A40000E949C070E94C0160E94E90A8BE08093C6
:101A50005A010E94D6239F938F9380E894E09F932E
:101A60008F930E943A060F900F900F900F900E9454
:101A7000F5069C012F3F9FEF390709F489C1211515
:101A8000310519F02F3F310569F40E94E10A0E94E7
:101A9000481988E794E09F938F930E943A060F902D
:101AA0000F9076C190915B01923009F451C018F407
:101AB000913041F06DC1933009F4CCC0943009F4F9
:101AC00047C066C190915701923099F028F499234C
:101AD00041F09130C1F039C0933061F1943081F11F
:101AE00034C0803E21F0813E51F482E005C081E0A7
:101AF00003C08D31D9F483E08093570149C187FF3A
:101B0000E3C08F770DC1863301F118F48A3229F4CE
:101B10001CC08A3AD1F0863BC1F087FD03C00E9409
:101B2000640A0BC08F770E94640A0DC08D3969F476
:101B300084E0E2CF853449F485E50E94D90905C0E7
:101B4000853C19F485E50E94F4091092570120C1E3
:101B5000E09156014E2F50E04930510508F077C012
:101B6000FA01E15FFE4F0C940B26803E69F030F4E1
:101B7000833871F0843871F48FE757C0813E31F0BB
:101B8000803F41F481E05BC082E059C084E057C0EF
:101B900082E04BC087FF98C00E94E10A8DE594E087
:101BA00098C0893509F453C0803F19F0823119F487
:101BB0004EC083E044C01092560187FD03C00E94CE
:101BC000100A82C00E94E10A83E594E082C0833853
:101BD00021F0843821F48FE738C082E036C01092BB
:101BE000560187FF9DC00E94E10A89E494E071C01C
:101BF00010925601823109F4CBC0893509F4C8C06E
:101C000087FD03C00E94100A8BC00E94E10A8CE38A
:101C100094E05FC0843121F0803FC9F486E00FC0BA
:101C200085E00DC0873799F480E00E94D9090FC084
:101C3000843169F487E003C0803F49F488E08093F1
:101C40005601A6C0873719F480E00E94F40910926B
:101C500056019EC090915501913009F443C038F06F
:101C6000923009F463C0933009F47FC091C0863884
:101C700009F168F48338D1F020F4803819F582E056
:101C80006CC08438A9F08538E9F48BE01DC08C382D
:101C9000A9F030F4873881F08B38A1F481E014C0CA
:101CA0008D3871F0803F71F481E057C082E00CC044
:101CB0008FE70AC086E008C080E006C089E004C063
:101CC0008AE002C087FD03C00E94D90961C08FE28B
:101CD00094E09F938F930E943A060F900F9010927A
:101CE0005A0156C0482F50E0FA01E358F109EB3091
:101CF000F10590F4E85EFE4F0C940B2682E045C09F
:101D00008FE743C08BE041C086E03FC081E03DC02B
:101D100089E03BC08AE039C01092550187FD03C0BD
:101D20000E94F40935C085E294E0D3CF853279F082
:101D300030F4863171F08E3199F480E00BC0863238
:101D400021F0803F69F483E008C08DE503C083E59E
:101D500001C081E50E94D90905C08093550118C0D2
:101D60000E94E10A1092550113C08E3169F020F4EF
:101D70008631B1F781E509C0853221F0863281F7DD
:101D80008DE503C083E501C080E00E94F409EACF3D
:101D900081E0DF91CF910895809193020895089595
:101DA000CF93DF9300D01F92CDB7DEB72091990378
:101DB000243021F523E029839B838A8382E080936A
:101DC000E9008FEF9091E800815095FD06C095EDF8
:101DD0009A95F1F700008111F5CF8091E80085FF19
:101DE0000DC040E050E063E070E0CE0101960E943B
:101DF0002C138091E8008E778093E8000F900F906D
:101E00000F90DF91CF910895CF93DF9300D01F9271
:101E1000CDB7DEB720919903243029F522E029833C
:101E2000805891099B838A832093E9008FEF9091DA
:101E3000E800815095FD06C095ED9A95F1F70000F8
:101E40008111F5CF8091E80085FF0DC040E050E0A2
:101E500063E070E0CE0101960E942C138091E800AF
:101E60008E778093E8000F900F900F90DF91CF91C5
:101E70000895CF93DF93EC0190919903943009F08A
:101E800048C0809114018823D9F0809115018823DE
:101E9000B9F09093E90081E8815049F09091E80011
:101EA00095FD05C09AE29A95F1F700C0F5CF8091B3
:101EB000E80085FF2EC040E050E060E270E019C00D
:101EC00081E08093E90081E8815059F09091E80029
:101ED00095FD07C0EFE3F1E03197F1F700C0000096
:101EE000F3CF8091E80085FF14C040E050E068E047
:101EF00070E0CE010E942C138091E8008E778093D1
:101F0000E80080E2FE01A3E7B2E001900D928A951D
:101F1000E1F7DF91CF910895CF93C0917101C11185
:101F20000BC00E94E223643C79408105910520F0BA
:101F300081E080937101C1E08C2FCF910895FF92D1
:101F40000F931F93CF93DF93D82F0FB607FE83C055
:101F500080919903843081F08091070190E001968F
:101F60002091090130E0822393232091080130E081
:101F70008217930709F0C9C00E948C0F811110C00D
:101F80008091070190E001962091090130E08223C1
:101F900093232091080130E08217930709F0B5C020
:101FA0000E94D6238C01C091E900CF709091EC0083
:101FB000892F817090FD80E8C82B83E08093E90031
:101FC00085E0F82E8091EB0085FD42C08091EB000A
:101FD00080FF3EC08091EE0087FF3AC080910801EB
:101FE00090910701981709F457C09091E80095FF68
:101FF0008AC0E0910501F0910601E80FF11D2081F2
:102000008F5F909109018923809308012093F1004B
:102010008091E80085FDE2CF8091E80080FFDECF6F
:102020008091E8008E778093E800F0920401D6CF8B
:102030008091070190E001962091090130E0822310
:1020400093232091080130E08217930709F448C0D8
:10205000CF70C093E90040910701842F90E0019672
:102060002091090130E0822393232091080130E080
:102070008217930709F44CC0E0910501F091060125
:10208000E40FF11DD083809107018F5F90910901CA
:102090008923809307013CC08091E80085FF33C00D
:1020A000D093F10081E09091F200992391F090910A
:1020B000E80090FF0EC09091E80095FF03C01092D9
:1020C000F100F9CF9091E8009E779093E800F092AC
:1020D0000401882309F4ACCFCF70C093E90018C085
:1020E00080910401882309F4B3CF0E94D6239C0178
:1020F0008017910711F4890165CF909104019150E7
:1021000090930401F8CF80E0CECF40910701B4CF87
:1021100080E0DF91CF911F910F91FF900895089576
:1021200042E061EC81E00E94A51242E061EC82E0B5
:102130000E94A51242E261EC83E00E94A51242E2F5
:1021400061EC84E00C94A51280919B03833009F428
:1021500055C030F4813071F0823009F48EC008959A
:102160008A3009F47AC08B3009F460C0893009F0F4
:102170009CC020C080919A03813A09F096C080915A
:10218000E800877F8093E80080919E0390919F03F1
:10219000892B21F460E283E792E003C060E080E0F5
:1021A00090E070E00E9479138091E8008B77809333
:1021B000E800089580919A03813209F076C08091F9
:1021C0009E0390919F03009719F0039709F06DC04B
:1021D0008091E800877F8093E8008091E80082FD8D
:1021E00005C0809199038111F8CF5FC08091F10003
:1021F000809393028091E8008B7753C080919A037B
:10220000813A09F052C080919E0390919F03892BDF
:1022100009F04BC08091E800877F8093E8008091AF
:10222000E80080FFFCCF8091140136C080919A03B2
:102230008132D9F580919E0390919F03892BA9F556
:102240008091E800877F8093E8000E94DA128091F5
:102250009C03809314010C94481980919A03813255
:1022600021F58091E800877F8093E8000E94DA12D0
:1022700080919D0380939402089580919A03813AFE
:10228000A1F48091E800877F8093E8008091E800C6
:1022900080FFFCCF809194028093F1008091E80050
:1022A0008E778093E8000C94DA120895809193025F
:1022B00080937201109293020E94E10A0C944819D3
:1022C0000C9456110E94832380919703882329F050
:1022D0000E94902381110C948F1208950E94A423D0
:1022E000809172018093930208950C946E11089569
:1022F0000C947711CF9384B7877F84BF0FB6F8947F
:10230000A8958091600088618093600010926000C1
:102310000FBE90E080E80FB6F89480936100909330
:1023200061000FBE8FE99FE00E9456238AE091E092
:102330000E94BB168BE295E00E94A1050E94CA0A8A
:102340000E946F170E9492150E94E51578940E94D2
:10235000711780919903843029F00E94A0160E9481
:102360007711F7CF89E195E00E94A1050E947811CD
:1023700087E095E00E94A105C3E080919903853034
:1023800019F40E946211F9CF0E9475172091E400A0
:102390003091E50080916F01909170012817390705
:1023A00009F464C08091E4009091E500909370017D
:1023B00080936F010E948C0F882309F457C080918D
:1023C0009903843009F052C08091E9008F70209108
:1023D000EC00922F917020FD90E8892BC093E900CA
:1023E0009091EB0090FF3FC09091EE0097FF3BC0B3
:1023F0009091080120910701291709F12091E80027
:1024000025FF1DC0E0910501F0910601E90FF11DC6
:1024100030819F5F209109019223909308013093AE
:10242000F1009091E80095FDE3CF9091E80090FFD6
:10243000DFCF9091E8009E779093E800D9CF9091FC
:10244000F200992381F09091E80090FF0CC09091E8
:10245000E80095FF03C01092F100F9CF9091E800D9
:102460009E779093E8008F708093E9000E94A016F9
:1024700084CF292F332723303105C9F060F4213070
:10248000310581F02230310509F041C084E790E048
:102490002BE835E040C021323105E1F02232310530
:1024A00031F135C082E190E02FEF35E034C099275B
:1024B0008130910549F028F0029749F5E1E4F5E013
:1024C00005C0E7E8F5E002C0E7E7F5E0849190E0B9
:1024D0009F0121C064307105D0F4660F771FFB01A6
:1024E000E05CFE4F2081318189E090E014C06430CF
:1024F000710568F4FB01EE0FFF1FE85CFE4F2081C1
:102500003181FB01EC5CFE4F808190E004C080E0F3
:1025100090E020E030E0FA0131832083089584E0E8
:1025200089BD86E089BD09B400FEFDCF8091D80049
:102530008F7D8093D8008091E00082608093E000DE
:102540008091E00081FDFCCF0895982F953068F5CB
:102550009093E900981739F07091EC002091ED000C
:102560005091F00003C0242F762F50E021FD02C0CF
:102570009F5FECCF3091EB003E7F3093EB003091CA
:10258000ED003D7F3093ED003091EB0031603093F2
:10259000EB007093EC002093ED005093F00020913D
:1025A000EE0027FDE5CF80E008958F708093E9006D
:1025B00081E0089580919A0387FF11C08091E8001F
:1025C00082FD05C0809199038111F8CF11C08091DF
:1025D000E8008B770BC080919903882349F08091A4
:1025E000E80080FFF8CF8091E8008E778093E800C4
:1025F00008952091E4003091E50095E64091EC00CB
:10260000842F817040FF23C08091E80080FD1DC0B1
:1026100080919903882399F0853099F08091EB009F
:1026200085FD11C04091E4005091E5002417350765
:1026300029F3915011F09A01E1CF84E0089582E0EE
:10264000089583E0089581E0089580E00895409121
:10265000E80042FFDDCF0895CF92DF92EF92FF9224
:102660000F931F93CF93DF93EC018B017A010E94AC
:10267000F912811135C0E114F10439F0F7018081BC
:102680009181081B190BC80FD91FC12CD12C011522
:10269000110529F18091E80085FD18C08091E800BE
:1026A0008E778093E8000E94A016E114F10449F0AF
:1026B000F70180819181C80ED91ED182C08285E048
:1026C0000FC00E94F912882311F30AC089918093E8
:1026D000F10001501109FFEFCF1ADF0AD8CF80E0D7
:1026E000DF91CF911F910F91FF90EF90DF90CF90EE
:1026F00008952091A0033091A1032617370748F0D1
:102700006115710539F42091E8002E772093E800D7
:1027100001C0B901FC0120E06115710561F18091F2
:1027200099038823D9F18530D9F18091E80083FDA0
:1027300039C08091E80082FD2BC08091E80080FFC5
:10274000EBCF8091F20090E06115710551F0883077
:10275000910538F421912093F1006150710901969F
:10276000F3CF21E0089709F020E08091E8008E7710
:102770008093E800D1CF2111D2CF0AC08091990374
:10278000882361F0853061F08091E80083FD0AC004
:102790008091E80082FFF2CF80E0089582E0089502
:1027A00083E0089581E008952091A0033091A10372
:1027B0002617370748F06115710539F42091E800B4
:1027C0002E772093E80001C0B901FC0120E06115DB
:1027D000710579F180919903882309F43DC0853012
:1027E00009F43CC08091E80083FD3AC08091E80084
:1027F00082FD2CC08091E80080FFE9CF8091F2003B
:1028000090E06115710559F08830910540F42491EC
:102810002093F1003196615071090196F2CF21E0C9
:10282000089709F020E08091E8008E778093E80017
:10283000CECF2111CFCF0AC080919903882361F0B8
:10284000853061F08091E80083FD0AC08091E80046
:1028500082FFF2CF80E0089582E0089583E008953A
:1028600081E008951F93CF93DF93CDB7DEB7AA978A
:102870000FB6F894DEBF0FBECDBFEAE9F3E080915A
:10288000F100819323E0E23AF207C9F70E94A41015
:102890008091E80083FF2EC180919A0390919B0361
:1028A000492F50E04A30510508F024C1FA01ED5D8E
:1028B000FE4F0C940B26803821F0823809F01AC1A3
:1028C00008C08091960390919703992389F08260C4
:1028D0000FC080919E038F70853008F00BC18093EC
:1028E000E9008091EB0085FB882780F91092E900D0
:1028F0009091E800977F9093E8008093F100109208
:10290000F100D1C0282F2D7F09F0F4C0882319F0E1
:10291000823061F0EFC080919C03813009F0EAC001
:10292000933009F080E0809397032EC080919C0340
:1029300081112AC080919E038F702FEF280F2430C1
:1029400008F0D8C08093E9002091EB0020FF1CC064
:10295000933021F48091EB00806214C09091EB00E1
:1029600090619093EB0021E030E0A90102C0440F98
:10297000551F8A95E2F74093EA001092EA00809191
:10298000EB0088608093EB001092E9008091E800F2
:10299000877F8093E8000E94DA12ACC08111AAC040
:1029A00010919C031F778091E3008078812B8093A6
:1029B000E3008091E800877F8093E8000E94DA12AC
:1029C0008091E80080FFFCCF8091E30080688093D5
:1029D000E300111102C082E001C083E080939903FB
:1029E00089C08058823008F085C080919C03909106
:1029F0009D038C3D53E0950779F583E08A838AE255
:102A000089834FB7F894DE01139620E03EE051E24F
:102A1000E32FF0E050935700E49120FF03C0E295CC
:102A2000EF703F5FEF708E2F90E0EA3010F0C796A6
:102A300001C0C0968D939D932F5F243149F74FBFFE
:102A40008091E800877F8093E8006AE270E0CE0121
:102A500001960E94791316C060919E0370919F03A6
:102A6000AE014F5F5F4F0E943912BC01892B09F400
:102A700041C09091E800977F9093E80089819A8106
:102A80000E94D4138091E8008B778093E80032C0D5
:102A9000803881F58091E800877F8093E8008091FD
:102AA00095038093F1008091E8008E7772CF8111B9
:102AB00021C080919C0390919D0399270297D4F4A3
:102AC0008091E800877F8093E80080919C03809349
:102AD00095030E94DA1280919503811106C08091BE
:102AE000E30087FD02C081E001C084E08093990388
:102AF0000E9490108091E80083FF0AC08091E80056
:102B0000877F8093E8008091EB0080628093EB00E8
:102B1000AA960FB6F894DEBF0FBECDBFDF91CF915E
:102B20001F9108950E94EF150E94F215E0EEF0E06B
:102B3000808181608083E8EDF0E080818F77808301
:102B400019BCE3E6F0E080818160808310929803F5
:102B500008950E94EF150E94F2158091D8008F779A
:102B60008093D8008091D80080688093D8008091AD
:102B7000D8008F7D8093D80084E089BD86E089BD30
:102B800009B400FEFDCF10929903109295031092A4
:102B900097031092960342E060E080E00E94A51245
:102BA0008091E1008E7F8093E1008091E20081605E
:102BB0008093E2008091E20088608093E20080913F
:102BC000E0008E7F8093E0000895E3E6F0E08081EE
:102BD0008E7F808381E0809398030C94A9151092D6
:102BE000E20008951092E10008951F920F920FB62F
:102BF0000F9211242F933F934F935F936F937F9383
:102C00008F939F93AF93BF93EF93FF938091E100D6
:102C100082FF0BC08091E20082FF07C08091E1003B
:102C20008B7F8093E1000E949F168091E10080FFDE
:102C300019C08091E20080FF15C08091E2008E7F74
:102C40008093E2008091E20080618093E2008091B5
:102C5000D80080628093D80019BC85E080939903E6
:102C60000E9460118091E10084FF30C08091E200F9
:102C700084FF2CC084E089BD86E089BD09B400FED4
:102C8000FDCF8091D8008F7D8093D8008091E100A6
:102C90008F7E8093E1008091E2008F7E8093E2003E
:102CA0008091E20081608093E20080919503882307
:102CB00011F084E007C08091E30087FD02C081E04D
:102CC00001C083E0809399030E9475118091E10017
:102CD00083FF24C08091E20083FF20C08091E10047
:102CE000877F8093E10082E080939903109295039F
:102CF0008091E1008E7F8093E1008091E2008E7FE1
:102D00008093E2008091E20080618093E20042E0E3
:102D100060E080E00E94A5120E948F10FF91EF9169
:102D2000BF91AF919F918F917F916F915F914F91E3
:102D30003F912F910F900FBE0F901F9018950895FF
:102D4000CF93809199038823A1F0C091E900CF70BF
:102D50009091EC00892F817090FD80E8C82B109233
:102D6000E9008091E80083FD0E943214CF70C09387
:102D7000E900CF91089590939A0280939902089563
:102D8000E0919902F0919A02309721F00190F08140
:102D9000E02D099480E00895EF92FF920F931F9326
:102DA000CF93DF93E0919902F0919A023097B1F1BD
:102DB0008C010280F381E02D099580918F0382FFC1
:102DC0002DC080FF04C088E097E00E94A105E801C3
:102DD00010E282E0E82E87E0F82E80918F0380FFDA
:102DE0000BC088811F928F93FF92EF920E943A0648
:102DF0000F900F900F900F90115021961111EDCF61
:102E000080918F0380FF0AC080E097E0DF91CF912F
:102E10001F910F91FF90EF900C94A105DF91CF913E
:102E20001F910F91FF90EF900895CF93DF93209122
:102E30009702309198022817390709F19093980268
:102E400080939702E0919902F0919A023097B9F03D
:102E5000EC010680F781E02D099580918F0382FFB8
:102E60000EC080FF0CC0DF93CF9382EF96E09F935C
:102E70008F930E943A060F900F900F900F90DF9162
:102E8000CF910895CF93DF932091950230919602D0
:102E90002817390709F19093960280939502E091E3
:102EA0009902F0919A023097B9F0EC010084F18513
:102EB000E02D099580918F0382FF0EC080FF0CC02A
:102EC000DF93CF9382EE96E09F938F930E943A0612
:102ED0000F900F900F900F90DF91CF9108950C9469
:102EE00018180E94CD230C94CE0ABF92CF92DF9285
:102EF000EF92FF920F931F93CF93DF9300D000D0F8
:102F00001F92CDB7DEB70E94F80A0CE912E0F12C4F
:102F10008F2D0E94DB0AB82EF801C080C82639F434
:102F2000F3940F5F1F4FF0E1FF12F2CF30C080919A
:102F30008F0381FD0E941918D12CEE24E3948C2D6F
:102F40008E21F9F0D982FA8291E08B2D8E2109F43D
:102F500090E09B830E94D6238160782F9D838C8391
:102F600049815A816B818D810E944F1849815A8114
:102F70006B817C818D810E946E23F80180818E257A
:102F80008083D394EE0CF8E0DF12D9CFC9CF8FEF56
:102F900089838A831B820E94D6238160782F9D8338
:102FA0008C8349815A816B818D810E944F180E94C8
:102FB0006D230E94C01690919B02891741F10E94D7
:102FC000C01680939B0290918F0392FF0EC090FFDA
:102FD0000CC01F928F9383E197E09F938F930E9481
:102FE0003A060F900F900F900F9080919B020F90D8
:102FF0000F900F900F900F90DF91CF911F910F9135
:10300000FF90EF90DF90CF90BF900C947F230F90B4
:103010000F900F900F900F90DF91CF911F910F9114
:10302000FF90EF90DF90CF90BF9008950C94E90A45
:103030000895EF92FF920F931F93CF93DF9389E24E
:1030400097E00E94A105C0E0D0E083E3E82E81E094
:10305000F82E0EE117E08C2F0E94DB0A0E945B2302
:10306000FF92EF921F928F93DF93CF931F930F9353
:103070000E943A0621968DB79EB708960FB6F8942F
:103080009EBF0FBE8DBFC031D10529F7DF91CF9113
:103090001F910F91FF90EF90089508950895CF9399
:1030A000DF93CDB7DEB72B970FB6F894DEBF0FBE18
:1030B000CDBF942F4F83252F588769877A878B87B9
:1030C0004A855B85452B31F02F3F31F481E09F3FEE
:1030D00019F403C081E001C080E080FD07C04F818A
:1030E000588569857A858B850E946E23DE0111964D
:1030F00086E0FD0111928A95E9F785E0FE01379699
:1031000001900D928A95E1F749815A816B817C810A
:103110008D819E810E945D1F2B960FB6F894DEBFB5
:103120000FBECDBFDF91CF910895CF93882309F4CF
:1031300065C0C82F8CEF8C0F813A20F080E58C0F92
:103140008E3248F48C2F0E94A725811157C08C2FF6
:103150000E9451220CC080E28C0F883058F4C77056
:1031600081E001C0880FCA95EAF70E94F622CF914C
:103170000C9430238BE58C0F833078F4C53A29F01A
:10318000C63A31F083E890E005C081E890E002C0E3
:1031900082E890E0CF910C94151788E58C0F873169
:1031A00068F5C83A89F0C93A91F0CA3A99F0CB3A31
:1031B000A1F0CC3AA9F0CD3AB1F0CE3AB9F0CF3A7D
:1031C000C1F080E090E017C082EE90E014C089EE7C
:1031D00090E011C08AEE90E00EC085EB90E00BC04D
:1031E00086EB90E008C083EB90E005C084EB90E0B4
:1031F00002C087EB90E0CF910C944217CF910895D5
:10320000882349F19CEF980F913A20F090E5980FB0
:103210009E3218F40E94A1220DC090E2980F9830BF
:1032200058F4877091E001C0990F8A95EAF7892FC9
:103230000E94FC220C9430239BE5980F933020F4DD
:1032400080E090E00C941517885A873120F480E0D4
:1032500090E00C9442170895882321F00E94F622F2
:103260000C9430230895882321F00E94FC220C94B2
:10327000302308950E9416230E94E5220E943023E5
:1032800080E090E00E94151780E090E00C944217D7
:103290000E9406230C943A19CF92DF92EF92FF928C
:1032A0000F931F93CF93DF9300D000D01F92CDB721
:1032B000DEB76C010E948123811101C385E0F60114
:1032C000DE01119601900D928A95E1F7F601408199
:1032D0005181238134812115310531F05F3F31F473
:1032E00081E04F3F19F403C081E001C080E080FD20
:1032F000E6C2F601F280E580E2948FE0E82249839D
:103300005A83FB82722F3D832C836F2D8D810E9407
:10331000C6218C010E94C5210E94B520E12FE295B3
:10332000EF708E2F90E0FC01E35DFE4F0C940B26B6
:10333000812F807F1F70882311F01295107FFF204E
:10334000B9F0112329F0812F0E9409230E94302314
:10335000802F0F900F900F900F900F90DF91CF91D3
:103360001F910F91FF90EF90DF90CF900C949518E4
:10337000802F0E940019112309F4A1C2812F0E94FD
:103380000F230F900F900F900F900F90DF91CF9120
:103390001F910F91FF90EF90DF90CF900C9430230E
:1033A000812F807F1F70803211F01295107F0023D3
:1033B00019F0013009F12BC0FF20A9F0EE2059F1DE
:1033C000F1E0812FEF1228C00F900F900F900F9017
:1033D0000F90DF91CF911F910F91FF90EF90DF90B1
:1033E000CF900C941923EE2021F021E0E21609F48D
:1033F00066C20E941C234DC0FF20E9F085E08E15B7
:1034000008F45DC20E94F322812329F042C0FF200C
:10341000F1F1E11015C0812F0F900F900F900F90D8
:103420000F90DF91CF911F910F91FF90EF90DF9060
:10343000CF900C942C1994E09E1508F440C229C03A
:10344000F601858180FF13C08F708583E4CF003F34
:1034500009F472C108F03EC180E4800F803208F4A4
:1034600042C1FF2009F4D3C1EE2009F483C1802FAB
:103470000E949518093309F0C3C1FFEF21EE84E0E3
:10348000F15020408040E1F700C0000018C2E11078
:10349000C0C1812F42C1812F86958695837019F016
:1034A0008130B9F00CC2FF2019F0C801937002C03E
:1034B00080E090E00F900F900F900F900F90DF91B1
:1034C000CF911F910F91FF90EF90DF90CF900C94D0
:1034D0001517FF2019F0C801937002C080E090E03A
:1034E0000F900F900F900F900F90DF91CF911F9141
:1034F0000F91FF90EF90DF90CF900C944217812FA7
:10350000837009F070C0F110DAC1202F2295269542
:103510002770220F220F602F6F70862F90E0A0E09F
:10352000B0E06C017D01022E04C0CC0CDD1CEE1C51
:10353000FF1C0A94D2F704FF12C08FE090E0A0E0D5
:10354000B0E004C0880F991FAA1FBB1F2A95D2F7AD
:10355000BC01CD01609570958095909503C060E0A9
:1035600070E0CB011695169513701230B1F040F54E
:103570006C297D298E299F29113031F10F900F90F0
:103580000F900F900F90DF91CF911F910F91FF90AF
:10359000EF90DF90CF900C94DA206C297D298E2952
:1035A0009F290F900F900F900F900F90DF91CF9168
:1035B0001F910F91FF90EF90DF90CF900C94F4202B
:1035C0000E94DA20C701B6010F900F900F900F9064
:1035D0000F90DF91CF911F910F91FF90EF90DF90AF
:1035E000CF900C94C020FF2019F0812F817001C072
:1035F0008695882309F463C1202F2295269527708C
:10360000220F220F602F6F70862F90E0A0E0B0E0B5
:103610006C017D01022E04C0CC0CDD1CEE1CFF1CD5
:103620000A94D2F704FF12C08FE090E0A0E0B0E06F
:1036300004C0880F991FAA1FBB1F2A95D2F7BC018F
:10364000CD01609570958095909503C060E070E025
:10365000CB011695169513701230B1F040F56C2918
:103660007D298E299F29113031F10F900F900F90F5
:103670000F900F90DF91CF911F910F91FF90EF90DE
:10368000DF90CF900C94A1216C297D298E299F2950
:103690000F900F900F900F900F90DF91CF911F918F
:1036A0000F91FF90EF90DF90CF900C94B3210E9488
:1036B000A121C701B6010F900F900F900F900F90AE
:1036C000DF91CF911F910F91FF90EF90DF90CF90FE
:1036D0000C948F21023F09F45EC008F449C0033FF7
:1036E00009F46CC0BECE902F9071E92E812F8F719E
:1036F000FF2051F00E942821802FEE2019F08295A2
:10370000807F8ACE8F7088CE0E944921802FEE2044
:1037100019F08295807F01C08F700F900F900F90ED
:103720000F900F90DF91CF911F910F91FF90EF902D
:10373000DF90CF900C943319FF20A9F0E4E0EE1550
:1037400008F4BDC0812F8F710F900F900F900F90D4
:103750000F90DF91CF911F910F91FF90EF90DF902D
:10376000CF900C946E21F5E0FE1508F4A8C0EACFC6
:10377000FF2099F0812F8F710F900F900F900F9075
:103780000F90DF91CF911F910F91FF90EF90DF90FD
:10379000CF900C942821FF2069F3812F8F710F9017
:1037A0000F900F900F900F90DF91CF911F910F917D
:1037B000FF90EF90DF90CF900C944921FF2089F08B
:1037C000812F8F710F900F900F900F900F90DF91BE
:1037D000CF911F910F91FF90EF90DF90CF900C94BD
:1037E00013210F900F900F900F900F90DF91CF91BA
:1037F0001F910F91FF90EF90DF90CF900C940E21CE
:10380000033509F43ACE073409F059C036CEEE201C
:1038100021F2802F0F900F900F900F900F90DF915B
:10382000CF911F910F91FF90EF90DF90CF900C946C
:103830000019412F4F70602FC6010E9442240F9043
:103840000F900F900F900F90DF91CF911F910F91DC
:10385000FF90EF90DF90CF900C94102001112FC0BB
:10386000FF2069F10E9448192FEF80E792E0215074
:1038700080409040E1F700C000000F900F900F9043
:103880000F900F90DF91CF911F910F91FF90EF90CC
:10389000DF90CF900C942324412F4F70602FC601EE
:1038A0000F900F900F900F900F90DF91CF911F917D
:1038B0000F91FF90EF90DF90CF900C9445240F90E4
:1038C0000F900F900F900F90DF91CF911F910F915C
:1038D000FF90EF90DF90CF9008951F93CF93DF93E9
:1038E00000D000D01F92CDB7DEB7942F4983252F8B
:1038F0005A836B837C838D834C815D81452B31F0B2
:103900002F3F31F481E09F3F19F403C081E001C0F3
:1039100080E0182F117080FD31C049815A816B8180
:103920007C818D810E94C621292F22952F702C30F9
:1039300030F42A30A0F42250223030F022C02C3053
:10394000C9F02F30B9F01DC0853A28F48430C0F496
:10395000823028F415C090E2980F983088F0883EA5
:1039600030F4803E68F48450813A58F409C0803FB6
:1039700041F406C093FB112710F903C010E001C009
:1039800011E0812F0F900F900F900F900F90DF910B
:10399000CF911F910895CF93DF9300D000D01F9255
:1039A000CDB7DEB70F900F900F900F900F90DF9173
:1039B000CF910895CF93DF9300D000D000D0CDB742
:1039C000DEB726960FB6F894DEBF0FBECDBFDF91EF
:1039D000CF910895CF93DF93C091AC028091AD0257
:1039E000C817A1F0D0E0CE0166E070E00E94FA2591
:1039F000FC01E255FD4F40815181628173818481D8
:103A000095810E94DA1C2196C770E8CFDF91CF9193
:103A100008954091DE025091DF026091E0027091C2
:103A2000E1028091E2029091E3020C94DA1C1F9370
:103A3000CF93DF938091E30282958F7009F05CC091
:103A40008091E002882309F457C02091AC021091C4
:103A5000AD02C091DE02D091DF02A091E102B091EF
:103A6000E20281E0CF3F09F080E0482F211709F4FE
:103A700043C0109721F0DF3F21F080E003C081E0D8
:103A800001C0842F30E080FD33C0C90166E070E0E2
:103A90000E94FA25FC01E255FD4F81818D1328C05B
:103AA00080818C1325C08281811122C08381948101
:103AB0008A1B9B0B883C9105D8F48091E3028F70A0
:103AC00080618093E302C90166E070E00E94FA25FC
:103AD000FC01ED54FD4F90819F70906190838EEDBD
:103AE00092E00E944C19DF91CF911F910C94EA1C37
:103AF0002F5F3F4F2770BACFDF91CF911F9108956D
:103B00009F92AF92BF92CF92DF92EF92FF920F936C
:103B10001F93CF93DF93CDB7DEB761970FB6F894BD
:103B2000DEBF0FBECDBF8C0185E0F801DE011D9622
:103B300001900D928A95E1F7F80140812181F28090
:103B4000C380D4809091DE023091DF026091E10267
:103B50007091E2026115710531F03F3F31F481E06F
:103B60009F3F19F403C081E001C080E0F82FF1709D
:103B70009F2E80FD59C18EEDA82E82E0B82EE090D8
:103B8000E002F601E61BF70BEE2009F4EDC0809190
:103B9000E302582F507FE83CF10508F0A7C051110F
:103BA00056C0231313C0491311C0EF2CF1100EC0DF
:103BB0008F7080618093E3020E94091DC5010E94FD
:103BC0004C198091E302F801858364C1C114D104CA
:103BD00031F02F3F31F481E04F3F19F403C081E011
:103BE00001C080E080FD03C081E08F2502C080E03D
:103BF00090E0F82FF170EF2E80FF1FC0E091AC0233
:103C00003091AD02E31709F421C1F0E0CF0166E085
:103C100070E00E94FA25DC01A255BD4F11968C91EF
:103C20001197281307C08C91481304C012968C91E9
:103C3000F81203C03196E770E5CFEF2CFF2009F4AE
:103C400029C18091E30281608093E30264C0231361
:103C500006C0491304C0F11002C0F801A9C04D8785
:103C60002E87FF867C2DD98AC88A522F6F2D89898D
:103C70000E946D1C8823A1F1FF2091F12091E302A5
:103C8000822F82958F7090E0029774F08091DE020F
:103C90009091DF0298878F831986DB86CA862C87EE
:103CA000CE0107960E944C1986E0F801AEEDB2E015
:103CB00001900D928A95E1F70E94171D0E94091D3F
:103CC00012C0231751F14D872E87FF867C2DD98A8C
:103CD000C88A522F6F2D89890E946D1C81112CC0BA
:103CE000C8010E944C19EE24E394D4C05111E9CFCD
:103CF0007C2DD98AC88A522F6F2D89890E94CB1CAE
:103D00008EED92E00E944C1986E0F50111928A95A1
:103D1000E9F70E94091DE12CBDC04913D4CFF11071
:103D2000D2CFF8018583C8010E944C1986E0F501C5
:103D300011928A95E9F7AEC0FF2091F22091E3023B
:103D4000822F82958F7090E002970CF4ADCF809116
:103D5000DE029091DF029A8389831B82DD82CC820E
:103D60002E83CE0101969ECFE83CF10508F04CC0B1
:103D7000EF2CFF2009F4B4CF231330C049132EC019
:103D80002091E30220FD21C0822F82958F70482F61
:103D900050E041155105C9F0F80125834F30510518
:103DA00041F08F5F982F9295907F822F8F70892B93
:103DB0008583C8010E944C1986E0F801AEEDB2E09F
:103DC00001900D928A95E1F72CC086E0F801AEEDE6
:103DD000B2E001900D928A95E1F75CC04D872E8785
:103DE000FF867C2DD98AC88A522F6F2D89890E941F
:103DF0006D1C811159CF8091E30281608093E302B1
:103E0000C8010E944C1946C07C2DD98AC88A522FFD
:103E10006F2D89890E94CB1C86E0F50111928A954D
:103E2000E9F70E94091D36C0FF2009F459CF4D87DC
:103E30002E87FF867C2DD98AC88A522F6F2D8989BB
:103E40000E946D1C882309F44BCF2ECF7C2DD98A7C
:103E5000C88A522F6F2D89890E94C621292F229549
:103E60002F70223028F49F7039F0811105C00BC0EB
:103E7000243028F49F7049F4805E883020F0C80117
:103E80000E944C199E2CE92C05C0F8019581907F69
:103E900099F7F9CF8E2D61960FB6F894DEBF0FBE5D
:103EA000CDBFDF91CF911F910F91FF90EF90DF90E9
:103EB000CF90BF90AF909F900895CF93DF93CDB7F1
:103EC000DEB72C970FB6F894DEBF0FBECDBF4F8381
:103ED000588769877A878B879C87CE0107960E94CF
:103EE000801D8823D1F09F8188852A853B85232BDF
:103EF00031F08F3F31F481E09F3F19F403C081E03E
:103F000001C080E080FD6FC04F81588569857A854A
:103F10008B859C850E94DA1C66C086E0FE01379680
:103F2000DE01119601900D928A95E1F7FF81E885F7
:103F30006A857B856115710531F0EF3F31F481E0D1
:103F4000FF3F19F403C081E001C080E080FD4BC059
:103F50008091AD0290E09C012F5F3F4F2770332787
:103F60004091AC0250E02417350709F443C0F983AF
:103F7000EA837D836C8366E070E00E94FA25DC01B1
:103F8000A255BD4F96E0FE01319601900D929A9593
:103F9000E1F72093AD020E94EA1C25C090E066E0A4
:103FA00070E00E94FA2582559D4F0E94801D882353
:103FB00071F18091AC0290E066E070E00E94FA2519
:103FC000FC01E255FD4F4081518162817381848102
:103FD00095810E94DA1C8091AC0290E00196877076
:103FE00099278093AC028091AC029091AD02891325
:103FF000D5CF0DC00E9448191092AD021092AC02AC
:10400000EEEDF2E086E0DF011D928A95E9F72C964D
:104010000FB6F894DEBF0FBECDBFDF91CF910895EC
:10402000DF92EF92FF920F931F93CF93DF93FC01E8
:10403000892B09F488C0E12CF12CDD24D394EF0105
:1040400021968491853709F460C058F4843708F0CC
:104050004EC0843008F068C08130D1F0823071F1F8
:1040600072C0883709F45BC050F4863709F453C036
:10407000873709F068C08E2D0E94032352C09CE749
:10408000980F903708F05FC08F770E9400194EC0DC
:104090008F010E5F1F4FFE01849190E2980F9830C0
:1040A00050F48770FD2D01C0FF0F8A95EAF78F2F1E
:1040B0000E94092315C00E94951814C08F010E5F3D
:1040C0001F4FFE01849190E2980F983068F487703A
:1040D000FD2D01C0FF0F8A95EAF78F2F0E940F2355
:1040E0000E943023E80122C00E940019FBCFCF01BB
:1040F0000296FE01C491CC2361F0EFE9FFE0319715
:10410000F1F700C00000C150F6CFCF010296FE01CA
:10411000F490EC010BC00E94F322E82E07C00E942D
:1041200006230E94302302C00E9495188F2D8823F9
:1041300041F0EFE9FFE03197F1F700C00000815056
:10414000F6CFFE017CCFDF91CF911F910F91FF90B1
:10415000EF90DF90089560936403709365038093FC
:104160006603909367030C947E230895609368031D
:104170007093690380936A0390936B030C947D237F
:104180000F931F93009168031091690320916A03B4
:1041900030916B03602B712B822B932B6093680300
:1041A0007093690380936A0390936B031F910F913F
:1041B0000C947D230F931F93009168031091690362
:1041C00020916A0330916B03602371238223932330
:1041D000609368037093690380936A0390936B0301
:1041E0001F910F910C947D230F931F9300916803EF
:1041F0001091690320916A0330916B036027712746
:1042000082279327609368037093690380936A03FE
:1042100090936B031F910F910C947D2360E070E0ED
:10422000CB010C94AB200F931F9341E050E060E072
:1042300070E08A019B0104C0000F111F221F331F71
:104240008A95D2F7C901B8011F910F910C94AB2048
:104250000F931F9341E050E060E070E004C0440F12
:10426000551F661F771F8A95D2F78091640390913E
:104270006503A0916603B09167038A019B01082B37
:10428000192B2A2B3B2BC901B8011F910F910C94BC
:10429000AB200F931F9341E050E060E070E004C05A
:1042A000440F551F661F771F8A95D2F7409550958A
:1042B000609570958091640390916503A091660369
:1042C000B09167038A019B01082319232A233B230A
:1042D000C901B8011F910F910C94AB200F931F934C
:1042E00041E050E060E070E004C0440F551F661FDD
:1042F000771F8A95D2F78091640390916503A0910E
:104300006603B09167038A019B01082719272A27B2
:104310003B27C901B8011F910F910C94AB200F935B
:104320001F930091640310916503209166033091FF
:104330006703602B712B822B932B1F910F910C9491
:10434000AB200F931F93009164031091650320919C
:1043500066033091670360237123822393231F91A7
:104360000F910C94AB200F931F9300916403109155
:1043700065032091660330916703602771278227C8
:1043800093271F910F910C94AB2008958F929F92C9
:10439000AF92BF92DF92EF92FF920F931F93CF9352
:1043A000DF9300D000D01F92CDB7DEB76B837C8344
:1043B0008D838A018C819D81892B31F01F3F31F4DF
:1043C00081E04F3F19F403C081E001C080E080FF2D
:1043D00003C080E090E054C08B81882309F43DC085
:1043E0008090640390906503A0906603B09067038B
:1043F0008091680390916903A0916A03B0916B0367
:10440000882A992AAA2ABB2A2FE1E22EF12CD5016B
:10441000C4010E2C04C0B695A795979587950A946C
:10442000D2F780FD06C081E0E81AF10880F7D12CB0
:1044300007C0DE2CB8018E2D0E944306019799F328
:10444000E12FF0E093E0EE0FFF1F9A95E1F7EC51BA
:10445000FD4FE00FF11DD0820CC0E12FF0E083E0B2
:10446000EE0FFF1F8A95E1F7EC51FD4FE00FF11DB4
:10447000D08009831A8369817A818D2D0E94430639
:104480000F900F900F900F900F90DF91CF911F9191
:104490000F91FF90EF90DF90BF90AF909F908F9023
:1044A000089590911401992379F190911501992320
:1044B00059F1982F9695969596959F31A1F0E09198
:1044C0001601F0911701E90FF11D877021E030E02E
:1044D000A90102C0440F551F8A95E2F7CA019181D4
:1044E000892B8183089590918F0390FF29C01F929B
:1044F0008F9384E597E09F938F930E943A060F90E5
:104500000F900F900F900895209116013091170190
:10451000F90132969FEF40E05191851789F09F3F56
:1045200019F4511101C0942F4F5F4E31A9F79F3FED
:1045300039F0F901E90FF11D97FDFA95828308958D
:10454000089590911401992381F190911501992377
:1045500061F1982F9695969596959F31A9F0E091E7
:104560001601F0911701E90FF11D877021E030E08D
:10457000A90102C0440F551F8A95E2F7CA01809530
:10458000918189238183089590918F0390FF1CC0AE
:104590001F928F9386E397E09F938F930E943A0632
:1045A0000F900F900F900F900895E0911601F091E9
:1045B00017019F01225E3F4F9281891301C0128231
:1045C0003196E217F307C1F7089581E090E0E0919A
:1045D0001601F0911701E80FF91F10820196803241
:1045E0009105A9F7089580918E03089590918E0307
:1045F000892B80938E030895809590918E03892353
:1046000080938E03089580938E03089510928E03F5
:10461000089590918D03892B80938D030895809543
:1046200090918D03892380938D03089510928D03BB
:10463000089580936C03089510926C0308958091FF
:10464000160190911701FC0131969C01205E3F4FAD
:1046500080E0919191118F5FE217F307D1F70895F0
:10466000E0911601F091170180918E038083E09113
:104670001601F0911701908180918D03892B808321
:1046800080916C03882361F0E0911601F09117018D
:104690009081892B80830E941F23811110926C03CB
:1046A00080911601909117010C94CC1690934F01B4
:1046B00080934E0108958295982F9373292F220F8E
:1046C000220F982F9C7C96959695922B892F857515
:1046D000880F9A7A9695892B08950895CF93DF9342
:1046E00000D000D01F92CDB7DEB70F900F900F9083
:1046F0000F900F90DF91CF910895089508950C9435
:10470000161880E0089583B7817F8C6083BF83B7DC
:10471000816083BF7894889583B78E7F83BF089527
:10472000CF930E944D180E94F80A0E944E18C0E0D4
:104730008C2F0E94DB0A811104C0CF5FC031C1F70A
:1047400001C081E0CF9108950E94E10A0C944819BC
:104750001F920F920FB60F9211248F939F93AF93D6
:10476000BF938091900390919103A0919203B09197
:1047700093034196A11DB11D8093900390939103E3
:10478000A0939203B0939303BF91AF919F918F91A8
:104790000F900FBE0F901F90189582E084BD93E09C
:1047A00095BD9AEF97BD80936E0008952FB7F8944A
:1047B0008091900390919103A0919203B091930303
:1047C0002FBF08952FB7F8946091900370919103D3
:1047D00080919203909193032FBF08959C014FB74E
:1047E000F8948091900390919103A0919203B091DD
:1047F00093034FBF821B930B089578941F920F92DF
:104800000FB60F9211248F939F93AF93BF93809114
:10481000900390919103A0919203B091930301961C
:10482000A11DB11D8093900390939103A0939203D7
:10483000B0939303BF91AF919F918F910F900FBE53
:104840000F901F9018950E949215F89487E797E7AC
:10485000909301088093000887E090EBDC0180933F
:10486000A2039093A303A093A403B093A5039CE099
:1048700088E10FB6F894A895809360000FBE9093DE
:104880006000FFCF80E090E008950895CF93C82F97
:104890001F928F9388E797E09F938F930E943A0629
:1048A00081E090E0A0E0B0E0BC01CD0104C0660F63
:1048B000771F881F991FCA95D2F70E94B6200F90C4
:1048C0000F900F900F90CF910C944819CF9387328F
:1048D000A8F58E3108F02BC1803109F49FC0F8F49F
:1048E000873009F464C0A8F4863009F024C18091AF
:1048F0008F03817F8E7F80938F038DE797E00E94E7
:10490000A10580E69AE00E94A10581E080939403CE
:104910004CC08B30F1F18E3009F46CC00CC1863183
:1049200009F4B0C020F4813109F4EDC004C189312B
:1049300009F491C08B3109F449C0FDC0883349F1B5
:1049400050F4893209F4F1C0853309F4EEC087329E
:1049500009F0F1C0EAC0833409F4E7C028F48A33CF
:1049600008F4E9C08953E4C0883409F0E4C00E9427
:1049700048198FE49AE00E94A1052FEF83ED90E3A0
:10498000215080409040E1F700C000000E942324A5
:104990000CC088E997E05CC086E39AE00E94A1051C
:1049A00080918F03816080938F03C1E0C9C08091A3
:1049B0008F03C82FC17080FFEFCF82E49AE00E947E
:1049C000A10580918F03817F8E7F3DC090918F03E1
:1049D00091FBCC27C0F981E0C827892FC0FB81F962
:1049E00080938F03CC2319F089E29AE027C08BE1F2
:1049F0009AE02EC090918F0392FBCC27C0F981E002
:104A0000C827892FC0FB82F980938F03CC2319F02C
:104A10008CE09AE013C08CEF99E01AC090918F035C
:104A200093FBCC27C0F981E0C827892FC0FB83F90D
:104A300080938F03CC2351F080EF99E00E94A10571
:104A400080918F03816080938F037AC083EE99E019
:104A50000E94A105AACF84ED99E00E94A1058EEAEB
:104A600099E00E94A10586E699E00E94A1058EE3E7
:104A700099E00E94A10582EF98E00E94A10586ECD2
:104A800098E0E6CF88EB98E00E94A1050E94C0164E
:104A90001F928F938EE998E09F938F930E943A061E
:104AA000809114011F928F9387E898E09F938F93D2
:104AB0000E943A06809194021F928F9384E798E0B7
:104AC0009F938F930E943A06809115011F928F93B6
:104AD00081E698E09F938F930E943A060E94E2231A
:104AE0009F938F937F936F938AE498E09F938F9324
:104AF0000E943A068DB79EB746960FB6F8949EBFB1
:104B00000FBE8DBF52CF0E944819C091150181E0A0
:104B1000C827C0931501CC2329F080E498E00E94B7
:104B2000A1050EC085E398E093CF80E001C08D51D0
:104B30000E9446243ACF83E398E00E94A105C0E09A
:104B40008C2FCF91089580E008950C94A325CF93E6
:104B5000C82F80919403882319F0813059F042C006
:104B6000E0911601F09117018081823261F0843466
:104B7000D9F509C0E0911601F091170180818232C8
:104B800011F0843461F48C2F0E94A525811104C09A
:104B90008C2F0E94662424C081E090E021C08C2FDD
:104BA0000E94A32581111BC0C43189F018F4CB30B9
:104BB00029F010C0C93259F0C83361F48DE797E08D
:104BC0000E94A10584E797E00E94A10508C0109209
:104BD00094030CC082E797E00E94A10507C081E022
:104BE000817006C01092940380E002C080E0F8CF8C
:104BF000CF9108950024552704C0080E591F880F2F
:104C0000991F009729F076956795B8F37105B9F764
:104C1000802D952F0895EE0FFF1F0590F491E02D44
:064C20000994F894FFCF97
:104C26000080FFFF0573010000FFCC0E390FCF0E89
:104C3600040FD00E01016D03415400585400544531
:104C4600524D494E414C004E4F4E450041545F5A1D
:104C56003135300040362239A2066C064A06110666
:0E4C66009D05B605CF05EF050008000400020D
:106800008800EA44E944E244040005000600070069
:10681000080009000A000B000C000D000E000F001C
:1068200010001100120013001400150016001700CC
:10683000180019001A001B001C001D001E001F007C
:10684000200021002200230024002500260027002C
:10685000280029002A002B002C002D002E002F00DC
:10686000300031003200330034003500360037008C
:10687000380039003A003B003C003D003E003F003C
:1068800040004100420043004400450046004700EC
:10689000480049004A004B004C004D004E004F009C
:1068A000500051005200530054005500560057004C
:1068B000580059005A005B005C005D005E005F00FC
:1068C0006000610062006300640065A185006700EC
:1068D000680069006A006B006C006D006E006F005C
:1068E0007000710072007300890087008A008B00BD
:1068F000E000E100E200E300E400E500E600E7007C
:106900000100010001000100EA4401000100E2442D
:106910000100010001000100460001004A004B0097
:10692000010001004700480001000100E9440100A6
:106930000100010001000100010001003A003B00DC
:106940003C003D003E003F0040004100420043004B
:10695000010035004C0039000100440045005200A0
:1069600049000100010050004F0029004D004E0079
:1069700051000100010001000100010001000100BF
:1069800001000100010001000100010001000100FF
:1069900001000100010001000100010001004D00A3
:1069A0004A004E004B0001000100010001000100FF
:1069B00001000100010001000100010001000100CF
:1069C00001000100010001000100010001000100BF
:1069D00001000100010001000100010001000100AF
:1069E0000100010001000100490001000100010057
:1069F000010001000100010001000100010001008F
:00000001FF
